:100000000C9479010C94A1010C94A1010C94C607E5
:100010000C94A1070C947C070C94A1010C94A101F1
:100020000C94A1010C94A1010C94A1010C94A101C8
:100030000C94A1010C94A1010C94A1010C94A101B8
:100040000C9432070C94A1010C9400070C94DA066E
:100050000C94A1010C94A1010C94A1010C94A10198
:100060000C94A1010C94A1014572726F723A2000A8
:1000700041726475436F756E7465722056322E300E
:1000800035002C20617667206C656E20002C206C7A
:1000900061737420617420004D20202066697273A2
:1000A0007420617420002052656A2000206D730066
:1000B0002920696E200020282B002C20636F756E8C
:1000C0007420002C206E6F206D696E206C656E00B0
:1000D0002066616C6C696E670020726973696E6777
:1000E00000206D73002C206D696E206C656E200001
:1000F0006368616E67650066616C6C696E6700724B
:100100006973696E67002C20694D6F64652000502B
:1001100043496E742070696E2000205374617274BC
:1001200065640000000008000201000003040700ED
:100130000000000000000000000000250028002B47
:100140000000000000240027002A0020004D206449
:100150006566696E65642070696E200000000000AD
:10016000230026002900416464496E7400496C6CC8
:100170006567616C206D6F646520666F72207069C1
:100180006E2073706563696669636174696F6E2060
:1001900000496C6C6567616C2070696E20737065D6
:1001A00063696669636174696F6E20000404040406
:1001B0000404040402020202020203030303030311
:1001C00001020408102040800102040810200102EE
:1001D000040810204D2072656D6F76656420005212
:1001E000656D496E7400496C6C6567616C2070695F
:1001F0006E2073706563696669636174696F6E20F0
:10020000002000200020004D20696E746572766128
:100210006C732073657420746F200073697A6500B5
:1002200020002061742000206C656E200020737413
:100230006172742000442070696E20004420707543
:100240006C736520686973746F72793A2000204D71
:10025000696C6C697365636F6E6473004D204E65E5
:100260007874207265706F727420696E20002000AF
:100270004D2070696E20004D206D696E20636F7592
:100280006E7420004D206D696E20696E7465727603
:10029000616C20004D206D617820696E7465727606
:1002A000616C20004D206E6F726D616C20696E7400
:1002B000657276616C20004D205374617475733AD9
:1002C000200048656C6C6F003A002F002C20002045
:1002D0004800204100204C00204600205800204EBD
:1002E000002054002052002044002043005200000F
:1002F000111111241FBECFEFD8E0DEBFCDBF11E03A
:10030000A0E0B1E0E8E4F3E202C005900D92A03471
:10031000B107D9F726E0A0E4B1E001C01D92AD3FDE
:10032000B207E1F711E0C9E7D1E004C02197FE016F
:100330000E949711C837D107C9F70E94D6080C94BC
:10034000A2110C940000CF92DF92EF92FF920F93D4
:100350001F93CF93DF936C017A018B01C0E0D0E053
:10036000CE15DF0589F0D8016D918D01D601ED9193
:10037000FC910190F081E02DC6010995892B11F4C3
:100380007E0102C02196ECCFC701DF91CF911F9172
:100390000F91FF90EF90DF90CF900895FC01918D29
:1003A000828D981761F0828DDF01A80FB11D5D96D7
:1003B0008C91928D9F5F9F73928F90E008958FEF45
:1003C0009FEF0895FC01918D828D981731F0828DF9
:1003D000E80FF11D858D90E008958FEF9FEF089550
:1003E000FC01918D228D892F90E0805C9F4F821BB4
:1003F00091098F739927089580E696E00E94F00195
:1004000021E0892B09F420E0822F0895FC01848DDE
:10041000DF01A80FB11DA35ABF4F2C91848D90E02E
:1004200001968F739927848FA689B7892C93A08909
:10043000B1898C9180648C93938D848D981306C0C0
:100440000288F389E02D80818F7D80830895EF926B
:10045000FF920F931F93CF93DF93EC0181E0888F7E
:100460009B8D8C8D981305C0E889F989808185FD65
:1004700024C0F62E0B8D10E00F5F1F4F0F73112756
:10048000E02E8C8DE8120CC00FB607FCFACFE8897D
:10049000F989808185FFF5CFCE010E940602F1CF58
:1004A0008B8DFE01E80FF11DE35AFF4FF0820B8F99
:1004B000EA89FB898081806207C0EE89FF896083B9
:1004C000E889F98980818064808381E090E0DF9110
:1004D000CF911F910F91FF90EF900895CF93DF93ED
:1004E000EC01888D8823C9F0EA89FB89808185FD2C
:1004F00005C0A889B9898C9186FD0FC00FB607FC8D
:10050000F5CF808185FFF2CFA889B9898C9185FFCD
:10051000EDCFCE010E940602E7CFDF91CF91089583
:1005200080E090E0892B29F00E94FC0181110C945D
:10053000000008953FB7F89480915D0190915E01AD
:10054000A0915F01B091600126B5A89B05C02F3F27
:1005500019F00196A11DB11D3FBFBA2FA92F982FE9
:100560008827820F911DA11DB11DBC01CD0142E064
:10057000660F771F881F991F4A95D1F708952FB7E7
:10058000F8946091590170915A0180915B019091AA
:100590005C012FBF08952F923F924F925F926F920E
:1005A0007F928F929F92AF92BF92CF92DF92EF9203
:1005B000FF920F931F93CF93DF9300D000D0CDB75E
:1005C000DEB7882E0E94BF02AB01BC01282D30E0AF
:1005D000F901EE0FFF1FE05AFE4FA591B4914C9028
:1005E0004C82F901EF53FE4F908094244082220FF9
:1005F000331FF901E25EFE4F0190F081E02D808112
:10060000982209F460C1880C880C880C212C312CAC
:10061000AA24A39487E4B82E81E090E0022C01C0C4
:10062000880F0A94EAF7292D282309F444C1182DCC
:10063000120D5C808521E1E009F4E0E0212F30E03B
:10064000D901A452BE4FF1E08C91833009F0F0E063
:10065000C901880F991F880F991FDC01AF59BE4F40
:10066000CD90DD90ED90FC902A013B014C185D0887
:100670006E087F0873016201A091FB02AF5FA09337
:10068000FB02A091FB02A43110F01092FB02A0919A
:10069000FB02B0E0A951BD4F1C931091FB02DC019D
:1006A000AF59BE4F4D905D906D907C9004E0109FCF
:1006B000D0011124A956BD4F4D925D926D927C924E
:1006C0001397A091FB0214E0A19FD0011124A95B14
:1006D000BD4FCD92DD92ED92FC921397A091FB025B
:1006E0006A2E712CAE2FAA25A98383010D5C1D4FA4
:1006F0004A2ED8014C92A091FB02B0E0A15EBD4F02
:1007000010E2512E5C92D901AC53BE4FAC91A13096
:1007100011F0EF13C9C03901660C771C7B826A8225
:100720008301045E1B4FD8014D905C90411451042D
:1007300009F4BAC0612C712CC414D504E604F70482
:1007400040F59C012F593E4FD9014D935D936D9318
:100750007C931397EF17A1F0AA81BB81A451BC4FE2
:100760002D913C9111972F5F3F4F11963C932E9303
:10077000E091FB02F0E0E15EFD4FB2E5B08394C092
:10078000E091FB02F0E0E15EFD4FA8E54A2E4082D9
:100790008BC0D901A05CBE4FEF1308C02C91E09133
:1007A000FB02F0E0E15EFD4FB0827CC0EC91EF1700
:1007B00009F461C0FC01EC5DFA4F40835183628310
:1007C0007383FC01E45AFC4F408051806280738047
:1007D00045284628472821F4408351836283738348
:1007E00089010C501E4F1B830A83F8011081FC0104
:1007F000EC53FB4F4080518062807380112351F095
:100800000FEF401A500A600A700A408251826282D9
:10081000738219C01FEF411A510A610A710A40829E
:10082000518262827382F901E455FB4F20812F5F70
:100830002083FC01EC57FA4F40835183628373831A
:10084000EA81FB81A082FC01E450FD4F4080518091
:1008500062807380C40CD51CE61CF71CC082D18258
:10086000E282F382E091FB02F0E0E15EFD4F33E4CF
:10087000432E408217C0FC01E450FD4F4080518060
:1008800062807380C40CD51CE61CF71CC082D18228
:10089000E282F382E091FB02F0E0E15EFD4F20E5B1
:1008A000522E508269806C92FC01EF59FE4F4083BA
:1008B0005183628373830FEF201A300A18E02116E8
:1008C000310409F0A9CE0F900F900F900F90DF9197
:1008D000CF911F910F91FF90EF90DF90CF90BF903D
:1008E000AF909F908F907F906F905F904F903F90D0
:1008F0002F900895E82FF0E0E455FE4FE491E25088
:10090000E13011F4865005C0877098E0E99F800DB2
:10091000112490E00895CF93DF93C0E7D0E0F0E09A
:10092000C138DF0731F0FE0184910E94EB07219668
:10093000F6CFDF91CF910895CF93DF93C8E6D0E053
:10094000F0E0CF36DF0731F0FE0184910E94EB0723
:100950002196F6CFDF91CF9108952F923F924F923B
:100960005F926F927F928F929F92AF92BF92CF923F
:10097000DF92EF92FF920F931F93CF93DF93CDB748
:10098000DEB727970FB6F894DEBF0FBECDBF8983C1
:10099000282E312CC101880F991F880F991F9F8322
:1009A0008E83FC01EC5DFA4FC080D180E280F38041
:1009B0008C010C571A4FF80180819181A281B3817B
:1009C000C81AD90AEA0AFB0AEE81FF81EC53FB4FF1
:1009D0004080518062807380F101E455FB4F80813B
:1009E00053014201881A9108A108B108EE81FF81E4
:1009F000E45BFB4F80819181A281B381881A990ABF
:100A0000AA0ABB0AC114D104E104F10469F40E94EA
:100A1000BF02F80100811181228133816B017C01C9
:100A2000C01AD10AE20AF30A8FE091E00E9462083C
:100A30002981622F70E080E090E04AE00E94FE078A
:100A400086E091E00E946208F101EC53FE4F808144
:100A5000823051F0833029F0813051F480EF90E002
:100A600005C08FEF90E002C087EF90E00E9462081F
:100A70008101000F111F9801245E3B4FF901808115
:100A80009181892B11F185EE90E02C833D830E94AA
:100A900062082C813D81F9016081718180E090E0E4
:100AA0004AE00E94FE0781EE90E00E946208F10198
:100AB000E452FE4F8081823029F0833051F489ED79
:100AC00090E005C080ED90E002C083EC90E00E94D1
:100AD00062088AEB90E00E946208C301B2010E94A2
:100AE0004F0886EB90E00E946208C501B4010E94A5
:100AF0004F0880EB90E00E946208C701B6010E9497
:100B00004F088CEA90E00E946208F801E45EFB4F17
:100B100080819181892BA9F086EA90E00E94620889
:100B2000F801E451FC4F60817181F801E454FC4FFD
:100B300080819181681B790B80E090E04AE00E94FF
:100B4000FE0781149104A104B10409F46EC00E944F
:100B5000F60788E990E00E946208EE81FF81E45A7E
:100B6000FC4F80819181A281B3810E811F810C5144
:100B70001A4FF801C080D180E280F380BC01CD0122
:100B80006C197D098E099F090E944F088DE890E03D
:100B90000E946208EE81FF81EC5DFA4F80819181B5
:100BA000A281B381F8010081118122813381BC01CE
:100BB000CD01601B710B820B930B0E944F08F894C0
:100BC000EE81FF81E450FD4F6081718182819381CC
:100BD000A50194010E945211789482E890E02C8340
:100BE0003D834A835B830E9462082C813D814A8158
:100BF0005B81CA01B90127960FB6F894DEBF0FBE1C
:100C0000CDBFDF91CF911F910F91FF90EF90DF90BB
:100C1000CF90BF90AF909F908F907F906F905F909C
:100C20004F903F902F900C944F0827960FB6F89452
:100C3000DEBF0FBECDBFDF91CF911F910F91FF900F
:100C4000EF90DF90CF90BF90AF909F908F907F906C
:100C50006F905F904F903F902F900895AF92BF920A
:100C6000CF92DF92EF92FF920F931F93CF93DF9378
:100C70000E94BF026B017C010E94F6070E948B0458
:100C80008AE191E00E94AD0844E456E0CCE4D4E06F
:100C9000ACE1B4E0ECEBAE2EE3E0BE2E04EE15E0EA
:100CA00080E090E0FA011192AF019C012C503E4F80
:100CB000F90110829C01220F331F220F331FB9014B
:100CC0006C537B4FFB011082118212821382BC0194
:100CD00064557B4FFB011082199219921992199257
:100CE000B9016C577A4FFB01C082D182E282F38254
:100CF000B9016C5D7A4FFB01C082D182E282F3823E
:100D00002F593E4FF901C082D182E282F3821D92B7
:100D10001D929C01220F331F24513C4FF901118277
:100D20001082F501119211925F01F801C192D192E6
:100D3000E192F1928F0101968831910509F0B2CFCD
:100D4000E0E6F1E0A591B4918C918093C101E2E6D7
:100D5000F1E0A591B4918C918093C201E4E6F1E0B9
:100D6000A591B4918C918093C3010E94BF02009120
:100D70000601109107012091080130910901DC0161
:100D8000CB01800F911FA21FB31F80935C0690932D
:100D90005D06A0935E06B0935F06DF91CF911F9131
:100DA0000F91FF90EF90DF90CF90BF90AF9008959C
:100DB0000E949D111F920F920FB60F9211242F9334
:100DC0003F934F935F936F937F938F939F93AF93D3
:100DD000BF93EF93FF9380E696E00E940602FF9197
:100DE000EF91BF91AF919F918F917F916F915F91A3
:100DF0004F913F912F910F900FBE0F901F9018951C
:100E00001F920F920FB60F9211242F938F939F93DF
:100E1000EF93FF93E0917006F09171068081E0916D
:100E20007606F091770682FD12C090818091790656
:100E30008F5F8F7320917A06821751F0E0917906C7
:100E4000F0E0E05AF94F958F8093790601C08081D8
:100E5000FF91EF919F918F912F910F900FBE0F9067
:100E60001F9018951F920F920FB60F9211242F9377
:100E70003F938F939F93AF93BF938091590190912C
:100E80005A01A0915B01B0915C013091580123E0BF
:100E9000230F2D3720F40196A11DB11D05C026E8B2
:100EA000230F0296A11DB11D209358018093590173
:100EB00090935A01A0935B01B0935C0180915D0116
:100EC00090915E01A0915F01B09160010196A11D1A
:100ED000B11D80935D0190935E01A0935F01B0937B
:100EE0006001BF91AF919F918F913F912F910F9092
:100EF0000FBE0F901F9018951F920F920FB60F9272
:100F000011242F933F934F935F936F937F938F930E
:100F10009F93AF93BF93EF93FF9382E00E94CB0226
:100F2000FF91EF91BF91AF919F918F917F916F91C1
:100F30005F914F913F912F910F900FBE0F901F9097
:100F400018951F920F920FB60F9211242F933F9373
:100F50004F935F936F937F938F939F93AF93BF93C1
:100F6000EF93FF9381E00E94CB02FF91EF91BF913D
:100F7000AF919F918F917F916F915F914F913F9131
:100F80002F910F900FBE0F901F9018951F920F92E8
:100F90000FB60F9211242F933F934F935F936F934C
:100FA0007F938F939F93AF93BF93EF93FF9380E0D3
:100FB0000E94CB02FF91EF91BF91AF919F918F91D2
:100FC0007F916F915F914F913F912F910F900FBE45
:100FD0000F901F901895E0916006F09161060190C6
:100FE000F081E02D682F80E696E0099442E050E021
:100FF0006CE371E080E696E00C94A3018F929F92DF
:10100000AF92BF920F931F93CF93DF93CDB7DEB70D
:10101000A1970FB6F894DEBF0FBECDBF19A2423024
:1010200008F44AE08E010F5D1F4F842E912CA12CF5
:10103000B12CA50194010E945211E62FB901CA01F9
:1010400001501109EA3014F4E05D01C0E95CD801F7
:10105000EC93232B242B252B61F70115110571F03F
:10106000F80101900020E9F73197AF01401B510BC7
:10107000B80180E696E00E94A30102C080E090E003
:10108000A1960FB6F894DEBF0FBECDBFDF91CF9112
:101090001F910F91BF90AF909F908F9008954AE05D
:1010A0000C94FE07CF93DF93BC0180E090E04AE010
:1010B0000E94FE07EC010E94F6078C0F9D1FDF9136
:1010C000CF9108950F931F93CF93DF938C01C0E0CE
:1010D000D0E0F801EC0FFD1F6491662371F0E09100
:1010E0006006F09161060190F081E02D80E696E0C7
:1010F0000995892B11F02196ECCFCE01DF91CF918C
:101100001F910F910895CF92DF92EF92FF92CF93AC
:10111000DF9397FF19C06B017C018DE20E94EB0702
:10112000EC0166277727CB016C197D098E099F0991
:101130004AE00E94FE078C0F9D1FDF91CF91FF9028
:10114000EF90DF90CF9008954AE0DF91CF91FF902C
:10115000EF90DF90CF900C94FE07CF93DF930E9427
:101160006208EC010E94F6078C0F9D1FDF91CF9162
:101170000895CF93DF934AE00E94FE07EC010E949E
:10118000F6078C0F9D1FDF91CF910895CF93DF93CA
:10119000BC01990F880B990B0E948308EC010E94F7
:1011A000F6078C0F9D1FDF91CF910895CF93DF93AA
:1011B000CDB7DEB7E2970FB6F894DEBF0FBECDBF56
:1011C000789484B5826084BD84B5816084BD85B522
:1011D000826085BD85B5816085BD80916E0081602E
:1011E00080936E00109281008091810082608093D4
:1011F00081008091810081608093810080918000D6
:101200008160809380008091B10084608093B10000
:101210008091B00081608093B00080917A008460FA
:1012200080937A0080917A00826080937A00809126
:101230007A00816080937A0080917A008068809340
:101240007A001092C100E0917006F091710682E080
:101250008083E0916C06F0916D061082E0916E063D
:10126000F0916F0683E3808310927806E091740614
:10127000F091750686E08083E0917206F091730626
:10128000808180618083E0917206F0917306808195
:1012900088608083E0917206F09173068081806897
:1012A0008083E0917206F091730680818F7D808348
:1012B0000E949A024B015C01F4EFCF2EDD24D394FF
:1012C000E12CF12C0E949A02DC01CB0188199909CA
:1012D000AA09BB09883E9340A105B10558F001E079
:1012E000C01AD108E108F10818EE810E13E0911E32
:1012F000A11CB11CC114D104E104F10419F77894C4
:101300000E942E0684E496E0E8E1CE2EC80EC8A620
:101310000E94BF026D877E878F87988B80E696E05C
:101320000E94F001892B09F4D4C380E696E00E9464
:10133000CE018C32C9F480911E02873008F0C9C3F7
:10134000E82FF0E0EE0FFF1FE45FFD4F20911C023D
:1013500030911D02318320838F5F80931E02109293
:101360001D0210921C02B5C390ED980F9A30B0F494
:1013700040911C0250911D029AE0949F9001959F0C
:10138000300D1124205331097901E80EF11C87FD3D
:10139000FA94F0921D02E0921C029BC39FE9980F01
:1013A0009A3108F096C3883609F47DC334F4813647
:1013B00071F0843609F483C17EC3823709F4A9C26F
:1013C000833709F4A9C2893609F075C3CFC1C0902B
:1013D0001E02EC2DF0E0EE0FFF1FE45FFD4F809149
:1013E0001C0290911D0291838083C394C0921E02BF
:1013F0000E94BF024B015C0100910C0210910D0292
:10140000802F0E947A047C01C8010197479748F415
:10141000F801EC5DFE4F8081882319F028E12E153C
:1014200040F40E949C0481E991E00E946208C80196
:10143000A8C6A80144555E4F3A01FA0124915EEF17
:10144000D52ED20E80910E0290910F02823091051E
:1014500079F08330910599F00197D9F00E949C04AE
:101460008DE691E00E946208C8010E94C6080FC084
:10147000F701FF27E452FE4F82E0808308C0F701A6
:10148000FF27E452FE4F83E0808363E003C062E005
:1014900001C061E0C80180549E4FFC017491F301CA
:1014A00024912223C1F030E0220F331FF901EF5BBA
:1014B000FE4FA591B491F901E95CFE4F459154911D
:1014C0003FB7F8942C91709527232C93DA012C9137
:1014D00072237C933FBFB2E0BC1508F054C020914A
:1014E000100230911102232B09F441C0F801ED5D87
:1014F000FE4F3491FC012491F30144914423B9F14E
:10150000332339F1333091F038F43130A9F03230EF
:1015100001F534B53F7D12C0373091F03830A1F07D
:101520003430B9F4309180003F7D03C030918000A9
:101530003F77309380000DC034B53F7734BD09C08C
:101540003091B0003F7703C03091B0003F7D3093C1
:10155000B000E42FF0E0EE0FFF1FE95CFE4FA59115
:10156000B4913FB7F8944C91242B2C933FBFF3E0F8
:10157000CF1649F020911202309113022115310546
:1015800021F061E002C020E030E0FC018491F30131
:101590006490662009F4B4C56A946A94E62DF0E07C
:1015A000EE0FFF1FE25EFE4F0190F081E02D908173
:1015B000892B80834091680081E090E001C0880F12
:1015C0006A94EAF7842B80936800A7015527FA01F3
:1015D000EC53FE4F6083CA01880F991FFC01E45E43
:1015E000FB4F31832083DA01AC5BB94F2C9130E0A3
:1015F0002017310709F451C02D2D30E0F901EE0F0D
:10160000FF1FE05AFE4F65917491FB016081F90163
:10161000EF53FE4F60830C93FA01EC50FE4F1082A3
:101620009A01220F331F220F331FF901EC53FB4F96
:101630001082118212821382FA01E455FB4F10824C
:10164000F901E45BFB4F1082118212821382F901CF
:10165000EC57FA4F80829182A282B382F901EC5D4D
:10166000FA4F80829182A282B382F901EC51FA4F43
:1016700080829182A282B382F901EF59FE4F80826B
:101680009182A282B382FC01E451FC4F118210824C
:10169000FC01E454FC4F118210828DE491E00E9421
:1016A0006208B801110F880B990B0E9483088BE424
:1016B00091E00E9462088E2D0E94AD0427C1109116
:1016C0001E02E12FF0E0EE0FFF1FE45FFD4F80915F
:1016D0001C0290911D02918380831F5F10931E0254
:1016E000E0900C02F0900D028E2D0E947A041123DE
:1016F00071F09701215031092731310540F4F7018C
:10170000EC5DFE4F2081222311F0893128F00E94E8
:101710009C0486EE91E032C5F701E054FE4F24911F
:10172000F701E455FE4FE491EE2309F4EEC4E250D4
:10173000AE2FB0E0AA0FBB1FA25EBE4F0D90BC91B2
:10174000A02D3C91209523232C932C912111E2C4B0
:101750003091680041E050E001C0440FEA95EAF79B
:10176000242F2095232320936800D4C480911E0247
:10177000E82FF0E0EE0FFF1FE45FFD4F20911C0209
:1017800030911D02318320838F5F80931E0284304D
:1017900038F40E949C048BE192E00E946208B6C07B
:1017A00020910C0230910D02C901019780319E40B9
:1017B00038F00E949C0480910C0290910D025BC055
:1017C000A8EEB3E00E9474116B017C0160930601E6
:1017D0007093070180930801909309010E94BF0252
:1017E000DC01CB018C0D9D1DAE1DBF1D00915C0663
:1017F00010915D0620915E0630915F06801791077B
:10180000A207B30770F40E94BF02C60ED71EE81EDF
:10181000F91EC0925C06D0925D06E0925E06F092E0
:101820005F0620910E0230910F02C90101978031AD
:101830009E4038F00E949C0480910E0290910F020D
:101840001AC0A8EEB3E00E94741160930A0170936D
:101850000B0180930C0190930D01209110023091A7
:10186000110221311EE0310748F00E949C04809152
:101870001002909111020E9452081DC1A8EEB3E01F
:101880000E94741160930001709301018093020122
:10189000909303018091120290911302909305019D
:1018A0008093040187E092E00E94620860910C023C
:1018B00070910D0280E090E04AE00E94FE0785E012
:1018C00092E00E94620860910E0270910F0280E027
:1018D00090E04AE00E94FE0783E092E00E946208E6
:1018E000609110027091110280E090E04AE00E9445
:1018F000FE0781E092E00E946208609112027091FE
:10190000130280E090E04AE00E94FE070E94F60782
:10191000D2C00E942E06CFC087EB92E00E946208E0
:101920000E948B040E94F60784EA92E00E946208FB
:101930006091060170910701809108019091090161
:101940000E94B90884E992E00E94620860910A014D
:1019500070910B0180910C0190910D010E94B908CA
:1019600084E892E00E946208609100017091010198
:1019700080910201909103010E94B90887E792E0EB
:101980000E94620880910401909105010E94520812
:1019900004E416E0F12CD801ED908D01EE2099F0D1
:1019A00080E792E00E9462086E2D70E080E090E097
:1019B0000E9483088EE692E00E9462088F2D0E94AA
:1019C000AD040E94F607F394B8E1FB12E4CF8CE576
:1019D00092E00E946208C0905C06D0905D06E090A4
:1019E0005E06F0905F060E94BF0297018601061B0B
:1019F000170B280B390BC901B8010E944F088EE460
:101A000092E00E9462080E94F6078CE392E00E9436
:101A1000AD080E94BF022B013C018091FB0290E0C7
:101A2000029664E170E00E943E116C01812C912CC1
:101A30005401E12CF12CC7018C0D9D1D64E170E077
:101A40000E943E118C011C01220C331C220C331C01
:101A5000E114F10409F498C3F101E956FD4F8081C6
:101A60009181A281B381F101E95BFD4F40815181F8
:101A700062817381840F951FA61FB71F8815990572
:101A8000AA05BB0508F080C3F101E956FD4F80802F
:101A90009180A280B3801FEFE11AF10A24E1E216DF
:101AA000F10449F608C00E94F6070E948B0482ECFC
:101AB00092E00E94AD0810921E0210921D02109238
:101AC0001C02ECE0F2E01192119232E0EC31F307EB
:101AD000D1F780915C0690915D06A0915E06B09171
:101AE0005F06CD84DE84EF84F888C81AD90AEA0A32
:101AF000FB0AF7FE2CC080910A0190910B01A09186
:101B00000C01B0910D014D855E856F857889481B6C
:101B1000590B6A0B7B0BA4EEB5E0E4E4F6E080E041
:101B20009191992369F00D911D912D913C911397FD
:101B30006A017B01C01AD10AE20AF30AF7FE81E0CA
:101B40001496D8A4DE12ECCF882309F4D6C20E94E2
:101B5000BF022B013C0104E416E01A8F098F04EE4A
:101B600015E01C870B870CE114E01A8709870CEB42
:101B700013E018870F830CE414E01A8309831D8A8D
:101B80001E8A1F8A188E212C312CA98DBA8DCD90DA
:101B9000BA8FA98FCB8ECC2009F477C2F89471014B
:101BA000EE0CFF1CEE0CFF1CFEA6EDA687010C57E9
:101BB0001A4F18AB0FA7D8012D913D914D915C9113
:101BC000298B3A8B4B8B5C8BF701EC5DFA4F408194
:101BD000518162817381F701EC53FB4F80809180CA
:101BE000A280B380F101E455FB4FFAABE9AB208151
:101BF00078946A017B0189899A89AB89BC89C81A62
:101C0000D90AEA0AFB0ACB82DC82ED82FE82A98134
:101C1000BA81CD90DD90ED90FC90CC8EDD8EEE8E75
:101C2000FF8E75016401C21AD108E108F1080C8D1C
:101C30001D8D2E8D3F8DC01AD10AE20AF30AD501FF
:101C4000C401801B910BA20BB30B8C8F9D8FAE8FA9
:101C5000BF8FAB85BC850D911D912D913C9108A343
:101C600019A32AA33BA300910A0110910B01209113
:101C70000C0130910D010CA31DA32EA33FA3D30192
:101C8000C201801B910BA20BB30B08A119A12AA1C1
:101C90003BA1801B910BA20BB30BB7FD55C08091EC
:101CA000040190910501A0E0B0E0C816D906EA064B
:101CB000FB0618F18091000190910101A0910201B1
:101CC000B09103010B811C812D813E81801791070A
:101CD000A207B30790F48091060190910701A091AB
:101CE0000801B09109010CA11DA12EA13FA18017EF
:101CF0009107A207B30709F05FC0F894EDA5FEA510
:101D0000EC5DFA4F4082518262827382EDA5FEA59E
:101D1000EC57FA4F4082518262827382F101E4559E
:101D2000FB4F10827894E981FA8180829182A282AD
:101D3000B382A301920189899A89AB89BC89281B46
:101D4000390B4A0B5B0B4EC0809106019091070145
:101D5000A0910801B091090193018201081B190BA0
:101D60002A0B3B0BD901C80108A119A12AA13BA14B
:101D7000801B910BA20BB30BB7FD87C180910401AF
:101D800090910501A0E0B0E0C816D906EA06FB066E
:101D900008F47BC18091000190910101A0910201A2
:101DA000B09103010B811C812D813E818017910729
:101DB000A207B30708F069C1A981BA818D929D92EB
:101DC000AD92BC921397F894EFA5F8A94083518384
:101DD00062837383A9A9BAA91C9278942B813C8150
:101DE0004D815E818DEE92E029A73AA74BA75CA7B3
:101DF0000E9462080B8D602F70E080E090E00E94EE
:101E000083088AEE92E00E946208C501B4010E9434
:101E10004F0887EE92E00E946208C701B6010E9457
:101E20004F0884EE92E00E9462086C8D7D8D8E8D4D
:101E30009F8D0E944F0881EE92E00E94620829A5C2
:101E40003AA54BA55CA5CA01B9010E944F088EEDC9
:101E500092E00E946208C301B2010E948308A98532
:101E6000BA858D919C91892B09F18BED92E00E94AE
:101E70006208C101880F991F8C0104511C4FF801A1
:101E800060817181AF81B8858D919C91681B790BC0
:101E900080E090E04AE00E94FE07F894F80180811B
:101EA0009181AF81B8858D939C9378942C8D3D8DD5
:101EB0004E8D5F8D232B242B252B09F453C088EDE9
:101EC00092E00E9462080DA51EA5045A1C4FF8015D
:101ED00080819181A281B381BC01CD0129893A8998
:101EE0004B895C89621B730B840B950B0E944F0816
:101EF00085ED92E00E9462086B817C818D819E81DC
:101F00000E944F08D8011D921D921D921C9213979A
:101F1000E985FA8580819181892B21F1F8940DA5BD
:101F20001EA504501D4FD8016D917D918D919C91FE
:101F3000A70196010E945211F801108211821282AB
:101F40001382789482ED92E029A73AA74BA75CA769
:101F50000E94620829A53AA54BA55CA5CA01B90152
:101F60000E944F088091FB0290E0029664E170E0CD
:101F70000E943E116C018FEC92E00E946208E12CFD
:101F8000F12C21E0C7018C0D9D1D64E170E00E94E1
:101F90003E115C01FC01E951FD4F808190E082150A
:101FA000930509F062C08501000F111F000F111F7A
:101FB00021111FC0F801E956FD4F80819181A28156
:101FC000B381F801E95BFD4F4081518162817381EA
:101FD000840F951FA61FB71F2D893E894F89588DE5
:101FE00082179307A407B507A0F18CEC92E00E943A
:101FF0006208F801E956FD4F80819181A281B38189
:10200000BC01CD0164197509860997090E948308EE
:102010008AEC92E00E946208F801E95BFD4F608162
:102020007181828193810E944F0888EC92E00E9426
:102030006208F501ED5CFD4F608170E080E090E0AA
:102040004AE00E94FE07F501E15EFD4F80810E949B
:10205000EB07F801E956FD4F80819181A281B381A0
:102060008D8B9E8BAF8BB88F20E09FEFE91AF90A1A
:10207000A4E1EA16F10409F085CF0E94F607EB858A
:10208000FC854082518262827382FFEF2F1A3F0AE1
:102090000B851C850C5F1F4F1C870B8709851A85D4
:1020A0000E5F1F4F1A8709870F8118850E5F1F4F1C
:1020B00018870F8309811A810C5F1F4F1A830983C8
:1020C00018E12116310409F060CD8091060190914C
:1020D0000701A0910801B0910901CD84DE84EF844D
:1020E000F8888C0D9D1DAE1DBF1D80935C069093DE
:1020F0005D06A0935E06B0935F060E94900208C939
:102100000E949C0486E691E0D4CC0E949C048FED52
:1021100091E0CFCC9C013327F901EC5BF94F1082A1
:10212000F901EC50FE4F1082C901880F991F880FEA
:10213000991FFC01EC53FB4F108211821282138213
:10214000F901E455FB4F1082FC01E45BFB4F108268
:10215000118212821382220F331FF901E45EFB4FBA
:1021600011821082F901E454FC4F11821082F901AE
:10217000E451FC4F1182108284ED91E00E946208CC
:10218000C7010E94C60897CC85E392E00E946208CE
:10219000F801E951FD4FE081F0E0EC5BF94F60811F
:1021A00070E080E090E04AE00E94FE078DE292E05D
:1021B0000E946208F101E956FD4F80819181A28160
:1021C000B381BC01CD0164197509860997090E9484
:1021D000830887E292E00E946208F101E95BFD4F0B
:1021E00060817181828193810E944F0882E292E036
:1021F0000E946208F801ED5CFD4F608170E080E0B4
:1022000090E04AE00E94FE0780E292E00E946208AD
:10221000F801E15EFD4F80810E94EB070E94F60706
:1022200033CCE0E6F6E01382128288EE93E0A0E081
:10223000B0E084839583A683B78382E191E09183A4
:10224000808385EC90E09587848784EC90E0978785
:10225000868780EC90E0918B808B81EC90E0938B73
:10226000828B82EC90E0958B848B86EC90E0978B50
:10227000868B118E128E138E148E089597FB072E67
:1022800016F4009407D077FD09D00E94831107FC53
:1022900005D03EF4909581959F4F08957095619576
:1022A0007F4F0895A1E21A2EAA1BBB1BFD010DC092
:1022B000AA1FBB1FEE1FFF1FA217B307E407F507F6
:1022C00020F0A21BB30BE40BF50B661F771F881FD2
:1022D000991F1A9469F760957095809590959B0168
:1022E000AC01BD01CF010895A29FB001B39FC00111
:1022F000A39F700D811D1124911DB29F700D811D32
:102300001124911D0895AA1BBB1B51E107C0AA1FF0
:10231000BB1FA617B70710F0A61BB70B881F991F86
:102320005A95A9F780959095BC01CD010895EE0FBF
:10233000FF1F0590F491E02D099481E090E0F8945E
:082340000C94A211F894FFCFE8
:10234800D007000001003075000060EA00000000BE
:1023580000002702A301F001CE01E2016E026B002A
:102368006C006D00000000030405060708090A0B4D
:102378000C0D0E0F10110000000000000D0A0000E7
:00000001FF
